:03000000021D736B
:0C1D730078FFE4F6D8FD7581E10200362F
:0100190022C4
:061A54008B2C8A2D892E67
:101A5A00751A027F48121BD8121DB8EF20E0F9ABA5
:101A6A002CAA2DA92E1209FB7873E6FE08E6FDEDD5
:011A7A00FF6C
:011A7B002248
:100FCE00434647002D53322D0052415445434C5257
:100FDE0020554E49544C4954455452494754524554
:100FEE00565354525453544F505A45524F424155F2
:100FFE004444464C5453415645525354205043207A
:10100E00205F3120735F3220735F35207331207380
:10101E00203220732035207320313020733330205E
:10102E007331206D2032206D2035206D203130201F
:10103E006D3330206D312068200000000100020069
:10104E0005000A001400320064012C025804B00B93
:10105E00B8177046508CA001020408103046656522
:10106E0074596172644D6574724F6666204F6E20BE
:10107E00204E6F2020596573204F66662054696D8F
:10108E0065416C7420547269674F666620547269AC
:09109E00675374727452656320FB
:101B380025E02447F582E43410F58322052EE52EAE
:101B4800C3940222A62EE52E75F004A42208F608F6
:041B5800F608F62273
:10177A00789376AB0876CD08760008760AE408F600
:10178A0008760108F6087664087640121B5508F6B2
:10179A0078A1F608760A08F608763C08F608761460
:0F17AA0008F608760F121B5578AE7605021B1451
:10197900751E1D751FC01216327894E664CD700469
:1019890018E664AB600312177A78ADE6FFF46003DA
:0F199900EF700478AD760178AEE6B4FF02760504
:0119A800221C
:0D1D4900C2AF7DC07C1DE4FF121C7ED2AF36
:011D5600226A
:101632007539FF851E3A851F3B753C00753D007567
:101642003E93E4FFAB39AA3AA93B8F82758300121D
:1016520009CEAB3CAA3DA93E8F82758300120A0DCA
:101662000FBF1CE078ACE6FFF46003EF700478ACC7
:021672007601FF
:011674002253
:101B14007D01E4FF121B9D121D49C2AF7F937B1C04
:101B24007DC07C1D121C88D2AF7F021218A7E4FD71
:041B3400FF021B9DF4
:10051000E4F52C7BFF7A0F79CE12173A7F0512187B
:10052000A7A297829650FAA2969219A297921AE5DC
:100530002C75F004A424D7F9740F35F0FA7BFF1260
:10054000173A7F051218A7852C2DE4F52E7BFF7A2C
:100550000F79D212173AE52CB40A0040030205DEE7
:10056000900567F82828730205850205DE0205A6B6
:100570000205AE0205B20205BA0205C20205C602B4
:1005800005CE0205D67F01EF121B387895E6FC08F0
:10059000E6FD7401936D7003E4936C70028F2E0F6F
:1005A000BF0FE40206647897E6F52E020687789876
:1005B000800278A0E6F52E0206A1789FE6F52E02CD
:1005C00006CF78A9800278AAE6F52E0206EC78AB71
:1005D000E6F52E02072178AEE6F52E020747E52C58
:1005E000652D600302052FA219309601B35013A2A6
:1005F00096921930960C052CE52CC3940D4003E41B
:10060000F52CA21A309701B350D4A297921A3097C2
:10061000CDE52CB40D0050C690061FF828287302B3
:10062000064602066F0206750206930206AD020632
:10063000C10206DA0206F702070F02073502075861
:1006400002075E020764052EE52EC3940F40037572
:100650002E01E52E121B38E493FF7401937895CF99
:10066000F608EFF6121B4E240BF9741002072A123B
:10067000145E0205DE052EE52EC394034003E4F567
:100680002E7897A62EE52E75F004A4246BF974102D
:1006900002072A121B444003E4F52E7898A62EE5A3
:1006A0002E75F004A42477F9741002072A121B4453
:1006B0004003E4F52E78A0121B4C2477F9741080C7
:1006C00069121B444003E4F52E789FA62EE52E7593
:1006D000F004A4247FF974108050052EE52EC394F5
:1006E000044003E4F52E78A9A62EE52E75F004A4A7
:1006F0002487F974108033052EE52EC3940340033C
:10070000E4F52E78AA121B4C2487F97410801B057F
:100710002EE52EC394044003E4F52E78ABA62EE517
:100720002E75F004A42497F9741035F0FA7BFF12AB
:10073000173A0205DE052EE52EC394064003E4F5C4
:100740002E78AEA62EE52E9010659375F018A4FFB6
:10075000AEF012128C0205DE12177A0205DE121BB1
:0A076000140205DE43A2080205DEC4
:0A1D8B004552415300444F4E4500FD
:101D08007895E6F54F08E6F55022E564AE63780667
:011D180022A8
:10120000C217C21878ADE6FFE4FCFDFEFB7A20F9B8
:10121000F8120A2F8F6A8E698D688C67E47B40FA1A
:10122000F9F8120ABA8E618F62E4F52DF52EC3E546
:101230002E9562E52D9561501CE52C64816016AFFA
:101240002EAE2D1219A9121C6A8F2C052EE52E70B8
:10125000DD052D80D9E52CB48108E52E152E700210
:10126000152DE52E65627004E52D6561700CD217B1
:10127000121D57E4F563F5648007852D63852E64A0
:0B128000E4F565F566754E80121D0850
:01128B002240
:1019A900C3EF9562EE95615024EF7806C333CE33C9
:1019B900CED8F9FD751A02EE7873F6CFEDCFEF08A0
:0D19C900F67F50121C28121DB8EF20E0F927
:0119D60022EE
:031C0E00CDEFCD4A
:101C1100751A02EE7873F6ED08F67F50121C281241
:061C21001DB8EF20E0F900
:011C2700229A
:101C6A00751A017F50121BD8121DB8EF20E0F978BF
:031C7A0073E6FF0F
:011C7D002244
:101C5500121C0EE4FFFE0FBF00010EBE0FF8BFA061
:041C6500F5121C6AEE
:011C69002258
:0618DD00CBEFCBCAEECAFE
:1018E300301703301827751A03EA7873F6EB08F6F6
:1018F30008EDF67F50121C28121DB8EF20E0F9E422
:0D190300FFFE0FBF00010EBE0FF8BFA0F5E4
:0119100022B4
:1016B800752F0075300075314EE4F52E121D12C3DA
:1016C80033CE33CED8F97C00252EFFEC3EFEAB2F6F
:1016D800AA30A931852E827583001209CEFD121811
:1016E800DD052EE52EC3940640D2756500756606A5
:0116F80022CF
:10138D008E2C8F2D121D12C333CE33CED8F9256678
:10139D00FFE5653EFEEEC0E0EFC0E0E52CFDD0E0E0
:1013AD00FFD0E0FE1218DD0566E5667002056512D8
:1013BD001D12C333CE33CED8F92566FFE5653EFE4B
:1013CD00AD2D1218DD0566E566700205650552E561
:1013DD005270020551C3E5669440E56594004017CF
:1013ED00E4F565F5660564E564700205639562E5EF
:0813FD006395614002D2172242
:10145E00E4F565F5667BFF7A1D798B12173AD21883
:10146E00E4F539F53AC3E53A9562E53995615021CF
:10147E00E53AAE397806C333CE33CED8F9F5668E5B
:10148E00657D81FF1218DD053AE53A70D805398081
:10149E00D4C2187BFF7A1D799012173AE4F563F5E2
:0714AE0064F565F566C21745
:0114B5002214
:10140500E4F539F53AF53BF53CC3E53C9562E53B3A
:1014150095615044E53A6481603EAF3CAE3B12199C
:10142500A9121C6A8F3AE53A64807022AF390539F2
:10143500FCFDFEFBFAF9120DA57F2C120016AE3B42
:10144500AF3CE4FCFDFBFAF9120DA5121DA8053C05
:08145500E53C70B5053B80B1D8
:01145D00226C
:0215A7008F397A
:1015A900E4F53AF53BF53CF53DC3E53D9562E53C8F
:1015B90095615030E53B6481602AAF3DAE3C12191C
:1015C900A9121C6A8F3BE53BB4800FE53A65397077
:1015D90007AF3DAE3C0219A9053A053DE53D70C985
:0415E900053C80C578
:0115ED0022DB
:1016F900121D0878A0E6F553E4F551F5521216B813
:1017090085636B85646C7F01121AA330021A78A372
:10171900E6FE08E6FFE4FCFD7B64FAF9F8120A2FFD
:101729008F608E5F8D5E8C5D300505C205121C3F92
:01173900228D
:1018330085632C85642DE56645656008052DE52DDA
:101843007002052C856B63856C641216B8852C6356
:10185300852D64C3E52D9562E52C95614007E4F57C
:0A18630063F564D2177F02021AA396
:101C7E00740478FF769612FF0322740078FF76962E
:041C8E0012FF03221C
:030033000210A711
:0D10A700C0E0C0F0C083C082C0D075D0088A
:1010B400E5D954F8FF120BD310E10810E11010F039
:1010C40018110B2010F228110B30110D3811134098
:1010D400110B48112C5011495800001157851DDA85
:1010E400C2DDC2DC751B00751C008070800EE51A21
:1010F40070028056051CE51C7002051B1200268F29
:10110400DAC2DDC2DC80558016D2DDC2DC804DC27D
:10111400DDC2DCE51A7004C2DA8041D2DA803DC255
:10112400DDD2DC7518048034AFDA121D7F051CE5AE
:101134001C7002051BC2DDC2DCE51A7004C2DA8031
:101144001BD2DA8017AFDA121D7FC2DDD2DC75182C
:0E115400028009751804C2DDC2DCD2DAC2DBEB
:0B116200D0D0D082D083D0F0D0E0329B
:101A020043910C43920CE4F5DBEF25E0F5DB301952
:101A12000343DB0175DD1775DC1775D84453F8FEF7
:091A220053F7FEE4F518D2E822A6
:101C2800E51830E002FF22E4F519751803EF25E006
:071C3800F51DD2DD7F022241
:101BD800E51830E002FF22E4F519151A751805EF2B
:0B1BE80025E04401F51DD2DD7F022244
:061DB80020DBFDAF182244
:0D002600151AAF19051974732FF8E6FF22A3
:0C1D7F0074732519F8EFF60519151A22E7
:101D1900E4F5847585FF53913FF592F5A475A5FF08
:011D29002297
:1019D700811902006F035D5733767E437F771004CA
:1019E700007B3E6C1F7C78773B020F382C5A1A6FAE
:0B19F700797518763C0E2F4E2B375DE3
:10186D004EFECCEFCC0F74732CF8EEF6EDC4332294
:10187D009019E7E493FF78D9F608EFF608F608F625
:10188D0022E493FF74D92EF8EFF60E22EE3395E095
:0A189D00FDFC227B007A0079D422C2
:10116D00E4FF0F2473F876CD0F74732401F87680A5
:10117D000F74732402F876E00F74732403F876F875
:10118D00301B0A0F74732404F87671800ACEEFCEEB
:10119D000F74732EF8767078D9E6FEC4540FFDCC1B
:1011AD00EFCC0F74732CF8EDF6EEC454F0FE78DA34
:1011BD00E6FD131313541F12186D54E0FE78DBE691
:1011CD00FD1313543F12186D3354C0FE78DCE6FD49
:1011DD00C31312186D33335480FECDEFCD0F7473DE
:1011ED002DF8EEF68F1A7F38121C28121DB8EF203D
:0211FD00E0F917
:0111FF0022CD
:10191100C21B12187D751A0A787376CD0876800875
:1019210076E00876F80876700876050876D50876A8
:101931009B0876FFE408F67F38121C28121DB8EFC9
:0319410020E0F9AA
:011944002280
:101BF300EF24F9600B14600C2402700EC21B8007E3
:0B1C0300D21B800312187D12116D220D
:1014B600C3EF648094E1400ED3EF648094FA500643
:1014C600EF24ACFF803CC3EF648094C1400ED3EFA1
:1014D600648094DA5006EF24CCFF8026C3EF648044
:1014E60094B0400ED3EF648094B9500674D02FFFA9
:1014F6008010BF2D047F0A8009BF5F047F0B800226
:031506007F0C2235
:101A7C00CEEDCECDEFCDCFEECF1214B6EF3395E049
:101A8C00FE74DB2FF58274193EF583E493FF74D951
:071A9C002DF8EFF602116DB9
:06173A008B3B8A3C893D57
:10174000E4FE9019E712188EBE04F7E4FEAB3BAA44
:101750003CA93D8E827583001209CEFF60191214D8
:10176000B6EFFD3395E0FC74DB2DF58274193CF582
:0A1770008312188EBE04D602116D1C
:04128C008F828E833C
:101290001218997B197AFC79FF78FFD3120B5A4008
:1012A0000390FC19AF82AE83121899E47B0F7A2762
:1012B000F9F8C3120B5A500390270FE4F52F74D49A
:1012C000252FF8E4F6052FE52FB405F2AE83AF82A3
:1012D0001218991218A0120DA578D7E6701A752F5A
:1012E0000374D3252FF8E6FF74D4252FF8EFF6D535
:1012F0002FEF78D4762080E11218A012173A300828
:101300000F7BFF7A1979D7121CF51218A0121CF561
:0113100022BA
:101CE200C214C216C213E4FDFF121B9DE4FD7F0164
:031CF200021B9D35
:101B9D00EF146011047016BD0104C2A78002D2A714
:0E1BAD00A2A7921522BD0103C2A622D2A62233
:101AA300EF24FE600D14601124027019D214756EB8
:101AB3000122C214A21592A722D216756F027D01CC
:061AC3007F01121B9D22B1
:101A2B00301412D56E0F30A707C2A7756E0F800545
:101A3B00D2A7756E23E56FD39400400CD56F09C206
:091A4B0016E4FD7F01121B9D222F
:101C920046554C4C005A4C4F470020332D340054CB
:041CA20072696700FC
:101AEF0078DEE6FE08E6FF22E6FE08E6FFE4FCFDF0
:101AFF002278CA120B9578C2020BAEC3E55C94B87C
:051B0F00E55B940B22D0
:03001300021B5C71
:101B5C00C0E0C0D075D010200F0CAF8DEFAD8BF561
:101B6C0058EDF559D20F758D00758B00D0D0D0E0A3
:011B7C003236
:0218A7008F3A76
:1018A900E4F53BF53CC3E53C953AE53B9400502310
:1018B900900000AF82AE83E4FCFD7B207A4EF9F8FC
:1018C900D3120B5A4003A380EA053CE53C70D605C8
:0318D9003B80D27F
:0118DC0022E9
:0E1D57007BFF7A1C799212173A7F0A0218A7B6
:0F1D3A00D20D301706121D57C20D221216F922B4
:05000E00C20D021833D1
:101C3F0078CE120BBA00000000121B0078CA120BEC
:061C4F00BA0000000022B3
:101D2A008E2C8F2DEEFF120016AF2DE52D02001618
:10003600121D19121D95121CE27F041218A7209793
:100046000B7D017F01121311D2AF80FE209612D2D2
:10005600AF121979C2197F70121A02121200120514
:1000660010121979120506D2AFC2197F70121A0240
:100076007F011218A71212001219117A1C79971211
:1000860004FB7A1C799C1204FB120019E4F5721227
:1000960017F87F011218A7E478D2F608F612001AAC
:1000A600A2969209A297920AE4F52478C6120BBA90
:1000B60000000000E4F52578CE120BBAFFFFD8F158
:1000C60078C2120BBA00000000C20B78CA120BBA33
:1000D60000000000C20EC212C20DE4F526F527C2CA
:1000E60008F55BF55CF558F559C20FF55AC210F5DF
:1000F60057F556F555F554F560F55FF55EF55DF582
:10010600207898E66004D2808002C28078A9E6242E
:10011600FE600B14600C2402700AD2018006D2061F
:100126008002D20078AAE624FE6007047006D20296
:100136008002D20778ABE624FE600B14600C240222
:10014600700AD2038006D2048002D205300117C29B
:100156000178A1121AF77B64FAF9F8120A2F8F5761
:100166008E568D558C54E572C3940240F9E4F572AF
:10017600A208B392A6209605209702D21130963592
:1001860030973230112FC21178C2120B95EC4D4EBA
:100196004F78CE700C120BBA00000000121B0080C4
:1001A60010120BBA0000000078C2120BBA00000051
:1001B60000D20AD209A209309601B3502AA2969219
:1001C6000930961C201119121B0A5014C201300B5B
:1001D60006C20B7F068004D20B7F07121BF3805BDF
:1001E600E4F55BF55C8054209651740A255CF55C59
:1001F600E4355BF55B121B0A4041E55C9410E55B58
:1002060094275037755B27755C10300807C20812B3
:1002160005068027D2087D01E4FF1213117F89129B
:1002260000167F011218A77F821200167F0112188E
:10023600A77F841200167F31120016A20A3097019A
:10024600B35017A297920A30971020110DB20D30B5
:100256000D05121D3A800312000E12076AAF57AE43
:1002660056AD55AC54EC4D4E4F602674FF2FF557E6
:10027600EE34FFF556ED34FFF555EC34FFF554AF8B
:1002860057AE56AD55FC4D4E4F7006200D03121D50
:100296003AAF60AE5FAD5EAC5DEC4D4E4F60237421
:1002A600FF2FF560EE34FFF55FED34FFF55EEC34BD
:1002B600FFF55DAF60AE5FAD5EFC4D4E4F70031255
:1002C600000E200F03020370C2AFC20FD2AFE48547
:1002D600592B85582AF529F528AF2BAE2AAD29AC1E
:1002E600287B107A27F9F8120A2F8F2B8E2A8D2950
:1002F6008C28E4FB7A90F9F81215EE8F2B8E2A8D56
:10030600298C28789FE66009C374B89FFF740B9EFA
:10031600FEE55A14601624FE602024037049C3EFDC
:1003260094B0EE9404500E755A018009D3EF9414DC
:10033600EE94054035755A038030C3EF94B0EE94C1
:10034600045027755A01300006200D03121D3A305D
:100356000305C203121C3F300D02D2107BFF7A1C2C
:1003660079A112173A8003E4F55A0525E525C394C9
:100376000150030204F5E4F525FB7A0079DD121A33
:100386005478DEEEF608EFF678DDE66402600302E6
:1003960004F578C6120BA1E8C0E0E9C0E0EAC0E0C7
:1003A600EBC0E0121AEF7897E6FD12155BD0E0FB82
:1003B600D0E0FAD0E0F9D0E0F8EB2FFFEA3EFEE914
:1003C6003DFDE83CFC78C6120BAE0524E524C3943B
:1003D6000550030204F578C6120B95E47B05FAF97D
:1003E600F81215EE78C6120BAE78C6120B9578C2C7
:1003F600120BA1C3EF9BFFEE9AFEED99FDEC98FC64
:1004060078C6120BAE78CE120B9578C6120BA1D316
:10041600120B5A400A78C6120B9578CE120BAE30E4
:100426000B0D78D0E6FF08E678E0CFF608EFF67811
:10043600C8E6FF08E678DECFF608EFF6300B0308CD
:10044600800278DEE6FE08E6FF12128C30120612F3
:100456001AEF121D2A0527E52770020526C378968E
:1004660096E52618964038E4F526F527300E06124E
:100476001AEF121D2A300D277F03121AA32017190F
:1004860078A0E6600C3010097F007E8212138DC2C0
:1004960010121AEF12138D8006121D5712000E78D5
:1004A600C6120B9578CA120BAE78C6120BBA0000AC
:1004B6000000E4F524300405C204121C3F30061681
:1004C60078A5121AF778CA120BA1D3120B5A400656
:1004D600200D03121D3A30071678A7121AF778CAAC
:1004E600120BA1C3120B5A5006300D0312000E1246
:0504F6001A2B02016C4D
:1004FB007BFF12173A7F041218A72278AEE6FDE4B1
:05050B00FF1213112294
:101AC900444C0021536967005A4C4F47004D4F441D
:101AD90000332D34004665622030372032303036ED
:061AE9000050524F4700BF
:10167500AF34AE33AD32AC31EC4D4E4F22EF24FFDB
:10168500F534EE34FFF533ED34FFF532EC34FFF588
:101695003122E475342075334EF532F53122E47587
:1016A5003401F533F532F53122752E00752F0075AD
:0316B5003093224D
:10076A00121D65EF7003020995121BBBEF120BD322
:10077A00095C2409672A098048096C5008B652079F
:10078A00A861083863098A68088B6C089172088E18
:10079A007308BA74092C7609277800000995C20BE8
:1007AA007BFF7A1A79C912173A121697121D65EF4A
:1007BA00700A121675600512168280F0121675708C
:1007CA0003020995121BBB8F2D1215A7E4F53412EB
:1007DA0016A7E47F06FEFDFCAB34AA33A932A83182
:1007EA00C3120B70501F121C6A8F2D120016E534AB
:1007FA002401F534E43533F533E43532F532E435A2
:10080A0031F53180CD121C6A8F2DE52D648060167A
:10081A00E52D64816010120016121C6A8F2D1200D9
:10082A0016752C018003E4F52CE52C70D8221216DB
:10083A00AE1216A3F52D1216756024121697121D04
:10084A0065EF700A121675600512168280F012168C
:10085A00756003120996052DE52DC3941C40D71225
:10086A001675601A7893B6AB0708B6CD0302096409
:10087A007BFF7A1A79CC12173A7F0A0218A7020963
:10088A0024B20E220214051216AEE4F52DAB2E0583
:10089A0030E530AA2F7002052F14F91209B5FF129C
:1008AA000016052DE52DC3941C40E22243A208221E
:1008BA00C20B752E00752F007530701216A3F52D18
:1008CA001216756024121697121D65EF700A121619
:1008DA0075600512168280F0121675600312099669
:1008EA00052DE52DC3940240D7121675602CAE7003
:1008FA00AF71EE3395E0FDFC78CA120BA1C3EF9BF2
:10090A00F538EE9AF537ED99F536EC98F535AF38B6
:10091A00789DE537F608EFF68040021632C20B02E0
:10092A00145E7A1A79D11209AA7A1A79D6121CF5A2
:10093A0078ACE62430FF120016121DA87F7612004A
:10094A00167A1A79DA1209AA7A1A79DE121CF502CB
:10095A001DA8C20BE4789DF608F6021B14C20B020E
:10096A00177AC20B7BFF7A1A79EA12173A7D017F4E
:10097A000112131180FE7D03E4FF121311D2122219
:0B098A0078AEE6FDE4FF121311C2126C
:1009950022121BBBAB2EAA2FA930852D8275830091
:1009A500EF120A0D227BFF121CF5121DA87BFF22F8
:0A1D9500E4F5955396BF53A27F2298
:1017F8005389F0438901538FFE758C70E4F58A5341
:10180800B8FD53B7FDD2A9D28C53890F43899053A1
:101818008FEFF58DF58B4391105392EF53B8F75333
:0B182800B7F7D2ABD28ED28AD2AA2230
:03000B00021D9F34
:091D9F000572758C70758A003222
:03001B00021DB112
:071DB100758D00758B0032F7
:101CA6000D0A003031323334353637383941424344
:041CB600444546005B
:101CBA00AF4DAB41AA42A943054D22AF40AE3FAD5D
:041CCA003EAC3D22CD
:101311005387BF75985053877FE4F5BABF010543E2
:10132100A240800353A2BFE4F5BDED146015146023
:101331001A14601F1460242404702575BEF075BF53
:101341000B802375BEF075BF05801B75BEF075BFA0
:1013510002801375BE7075BF01800B75BEB080032E
:1013610075BE30E4F5BF75BD035391FE4392014351
:1013710091025392FDC21C53B8EF53B7EF43B8101B
:0C138100E478C0F618F678C1F6D2AC2271
:030023000219457A
:10194500C0E0C0D075D01030981E78C0E6C3940FA3
:10195500501418E60624AFF8A69978C00618E6C311
:10196500941040027600C298309904C299C21CD0E6
:04197500D0D0E032BC
:08000300201CFDD21C8F992284
:101B7D0078C0E6D39400401508E60624AFF8E6FFDA
:0F1B8D0078C01608E6C394104005E4F6227F00E6
:011B9C002226
:03001600020003E2
:101BBB007F207E4E78C0E67010D3EF9400EE940039
:0C1BCB004007EF1F70EE1E80EB121B7D28
:011BD70022EB
:101CF5001209B5FF600C120016740129F9E43AFACD
:031D050080EE224B
:0E1D650078C0E6D3940040037F01227F002265
:091DA8007BFF7A1C79A6021CF5F0
:0E0DA5008F408E3F8D3E8C3D8B418A428943AC
:100DB300E4F54DEC4D4E4F7017E94A4B70057F300B
:100DC300020016121CBA8F827583007430020EC89B
:100DD300121CC7EC33502AE5434542454170077F57
:100DE3002D120016800D121CBA8F82758300742D8C
:100DF300120A0D121CC5120B4C8F408E3F8D3E8C78
:100E03003D754C017547007546CA75459A75443B57
:100E1300E4FFFEFDFCAB47AA46A945A844D3120B49
:100E2300705003020EB3121CC5A844120ABA8F4BAA
:100E33008E4A8D498C48EC4D4E4F7004E54C70231F
:100E4300E54B2430FFE5434542454170051200164A
:100E5300800EAE4D121CBC8E82758300EF120A0DFC
:100E6300E4F54CAF47AE46AD45AC44AB4BAA4AA9FB
:100E730049A848120A2FC8ECC8C9EDC9CAEECAC3AB
:100E8300E5409FF540E53F9AF53FE53E99F53EE5A0
:100E93003D98F53DAF47AE46AD45AC44E47B0AFA19
:100EA300F9F8120ABA8F478E468D458C44020E1309
:100EB300E542454345416010AB41AA42A943854DF4
:080EC30082758300E4120A0DA0
:010ECB002204
:100BF9000134C35001DBBF68028BBB800344B79843
:100C09000407B3B004D5AFC805A9ABE00689A7F8B6
:100C19000775A410086DA02809719C400A8198588D
:100C29000B9F94700CCA90880DE98CF90E048CA066
:100C39000EA88AAC0F4D88B80FF786C410A184D0CE
:100C4900115182DC120580E812BB7EF413747D0019
:100C590014307B0C14F2791815B877241680753086
:100C6900174B733C1819714818ED6F5419C46D600E
:100C79001AA16B6C1B7E69781C6167841D4A65909B
:100C89001E37639C1F2561A8201A5FB421125DC01D
:100C9900220D5BCC230E59D8241557E4251F55F096
:100CA900262F53FC27425208285B501429764E20E0
:100CB9002A9B4C2C2BC04A382CEE48442E1E4650F9
:100CC9002F55445C308F426831D1407433173E80D0
:100CD90034633C8C35B13A98370938A4386636B054
:100CE90039C734BC3B2D32C83C9D30D43E0F2EE071
:100CF9003F882CEC41062AF8428D29044418271014
:100D090045AB251C4741232848E121344A861F4029
:100D19004C311D4C4DE21B584F9C1964515D1770A5
:100D29005323157C54EF138856C4119458A20FA06D
:100D39005A830DAC5C6D0BB85E6009C4605807D06E
:100D4900625A05DC646203E8667301F4688A00008C
:100D59006AA1FE0C6CB8FC186ECFFA2470E6F83064
:100D6900000000000000000000000000000000007A
:100D7900000000000000000000000000000000006A
:100D8900000000000000000000000000000000005A
:0C0D99000000000000000000000000004E
:1017B90075F004E533A424F9F582E5F0340BF583DB
:1017C900E49322FE740193FF75F004E533A422F536
:1017D90083C37401939FFFE4939EFEE4228F348EAA
:0F17E900338D328C31228F308E2F8D2E8C2D220E
:101CCE00C3EF9DEE9C400AD3EF9BEE9A50037F012B
:041CDE00227F00223F
:040ECC008E318F32A2
:100ED000E4F5331217B9FC740193FD1217D124FD08
:100EE000F582E5F0340BF583E493FA740193FBAFDC
:100EF00032AE31121CCEEF7003020FBC1217B912C2
:100F000017CC24FDF582E5F0340B1217D88F378EFD
:100F100036F535F5341217D124FFF582E5F0340BA0
:100F2000F583E4931217CC24FBF582E5F0340B1221
:100F300017D88F3B8E3AF539F538AD39AC38120BEE
:100F40004C8F3B8E3A8D398C38AE31AF32E4FCFD9C
:100F5000EEC0E0EFC0E01217B9FE740193FBCAEED9
:100F6000CAD0E0FFD0E0FEC3EF9BFFEE9AFEED9407
:100F700000FDEC9400FCAB3BAA3AA939A838120A50
:100F80002FAB37AA36A935A8341215EEC8ECC8C95C
:100F9000EDC9CAEECACBEFCB1217D124FBF582E51F
:100FA000F0340BF583E493FE740193FFE4FCFDEB56
:100FB0002FFFEA3EFEED39FDEC38FC220533E53328
:0D0FC000C3946A5003020ED3E4FFFEFDFC53
:010FCD002201
:01001A0022C3
:101509001217E6AB34AA33A932A831E8C0E0789BB8
:10151900E6FE08E6FFE4FCFDD0E0F8120A2F1217F8
:10152900E6780E120B811217E6789DE6FE08E6FFB3
:10153900EE3395E0FDFCE5342FF534E5333EF53324
:10154900E5323DF532E5313CF531AF34AE33AD32FC
:02155900FC2272
:02155B008D2CD5
:10155D00120ECC1217EF1215091217EFE52C1460AD
:10156D001C14702DE47FE87E03FDFCAB30AA2FA97F
:10157D002EA82D120A2FE47BE87A0B800CAF30AE2B
:10158D002FAD2EAC2DE47B03FAF9F81215EE1217E0
:09159D00EFAF30AE2FAD2EAC2DE6
:0115A6002222
:1009B500BB010689828A83E0225002E722BBFE0240
:0909C500E32289828A83E4932273
:1009CE00BB010CE58229F582E5833AF583E02250DE
:1009DE0006E92582F8E622BBFE06E92582F8E22228
:0D09EE00E58229F582E5833AF583E4932242
:1009FB00BB010689828A83F0225002F722BBFE01DB
:020A0B00F322D4
:100A0D00F8BB010DE58229F582E5833AF583E8F01F
:100A1D00225006E92582C8F622BBFE05E92582C8CB
:020A2D00F222B3
:100A2F00E88FF0A4CC8BF0A42CFCE98EF0A42CFC66
:100A3F008AF0EDA42CFCEA8EF0A4CDA8F08BF0A4E4
:100A4F002DCC3825F0FDE98FF0A42CCD35F0FCEB43
:100A5F008EF0A4FEA9F0EB8FF0A4CFC5F02ECD3908
:0F0A6F00FEE43CFCEAA42DCE35F0FDE43CFC2275
:100A7E0075F008758200EF2FFFEE33FECD33CDCC2F
:100A8E0033CCC58233C5829BED9AEC99E5829840B2
:100A9E000CF582EE9BFEED9AFDEC99FC0FD5F0D68F
:100AAE00E4CEFBE4CDFAE4CCF9A88222B800C1B9B9
:100ABE000059BA002DEC8BF084CFCECDFCE5F0CBF7
:100ACE00F97818EF2FFFEE33FEED33FDEC33FCEB30
:100ADE0033FB10D703994004EB99FB0FD8E5E4F9EB
:100AEE00FA227818EF2FFFEE33FEED33FDEC33FCD8
:100AFE00C933C910D7059BE99A4007EC9BFCE99ACC
:100B0E00F90FD8E0E4C9FAE4CCFB2275F010EF2F10
:100B1E00FFEE33FEED33FDCC33CCC833C810D70710
:100B2E009BEC9AE899400AED9BFDEC9AFCE899F84B
:0E0B3E000FD5F0DAE4CDFBE4CCFAE4C8F922DE
:1015EE00C2D5E830E70FB2D5E4C39BFBE49AFAE428
:1015FE0099F9E498F8EC30E717B2D5121624120ACE
:10160E00BAE4C39BFBE49AFAE499F9E498F88003F0
:10161E00120ABA30D50DE4C39FFFE49EFEE49DFD91
:04162E00E49CFC221A
:0E0B4C00C3E49FFFE49EFEE49DFDE49CFC22BA
:100B5A00EB9FF5F0EA9E42F0E99D42F0EC6480C812
:060B6A0064809845F022B2
:100B7000EB9FF5F0EA9E42F0E99D42F0E89C45F0DB
:010B80002252
:100B8100E86010ECA2E713FCED13FDEE13FEEF138A
:040B9100FFD8F02277
:0C0B9500E6FC08E6FD08E6FE08E6FF228C
:0D0BA100E6FB08E6F908E6FA08E6CBF822C4
:0C0BAE00ECF608EDF608EEF608EFF62273
:100BBA00D083D082E493F608740193F60874029302
:090BCA00F608740393F674047339
:100BD300D083D082F8E4937012740193700DA3A3B1
:100BE30093F8740193F5828883E4737402936860C5
:060BF300EFA3A3A380DFC5
:00000001FF
